 NotifyFramePopStressTest

 Timestamp is e723598a (reproducible build file hash)

 Preferred load address is 0000000180000000

 Start         Length     Name                   Class
 0001:00000000 00001d70H .text$mn                CODE
 0001:00001d70 00000036H .text$mn$00             CODE
 0001:00001da6 00000092H .text$x                 CODE
 0002:00000000 000001a0H .idata$5                DATA
 0002:000001a0 00000038H .00cfg                  DATA
 0002:000001d8 00000008H .CRT$XCA                DATA
 0002:000001e0 00000008H .CRT$XCZ                DATA
 0002:000001e8 00000008H .CRT$XIA                DATA
 0002:000001f0 00000008H .CRT$XIC                DATA
 0002:000001f8 00000008H .CRT$XIZ                DATA
 0002:00000200 00000008H .CRT$XLA                DATA
 0002:00000208 00000008H .CRT$XLZ                DATA
 0002:00000210 00000008H .CRT$XPA                DATA
 0002:00000218 00000008H .CRT$XPZ                DATA
 0002:00000220 00000008H .CRT$XTA                DATA
 0002:00000228 00000008H .CRT$XTZ                DATA
 0002:00000230 00000000H .gehcont$y              DATA
 0002:00000230 00000000H .gfids$y                DATA
 0002:00000230 00000ed0H .rdata                  DATA
 0002:00001100 00000000H .rdata$CastGuardVftablesA DATA
 0002:00001100 00000000H .rdata$CastGuardVftablesC DATA
 0002:00001100 00000028H .rdata$T                DATA
 0002:00001128 0000008cH .rdata$voltmd           DATA
 0002:000011b4 0000032cH .rdata$zzzdbg           DATA
 0002:000014e0 00000008H .rtc$IAA                DATA
 0002:000014e8 00000008H .rtc$IZZ                DATA
 0002:000014f0 00000008H .rtc$TAA                DATA
 0002:000014f8 00000008H .rtc$TZZ                DATA
 0002:00001500 00000004H .tls                    DATA
 0002:00001504 00000004H .tls$                   DATA
 0002:00001508 00000008H .tls$ZZZ                DATA
 0002:00001510 00000200H .xdata                  DATA
 0002:00001710 0000020cH .edata                  DATA
 0002:0000191c 00000064H .idata$2                DATA
 0002:00001980 00000018H .idata$3                DATA
 0002:00001998 000001a0H .idata$4                DATA
 0002:00001b38 00000448H .idata$6                DATA
 0003:00000000 00000050H .data                   DATA
 0003:00000050 000007b8H .bss                    DATA
 0004:00000000 000002acH .pdata                  DATA

  Address         Publics by Value              Rva+Base               Lib:Object

 0000:00000000       __AbsoluteZero             0000000000000000     <absolute>
 0000:00000000       ___safe_se_handler_count   0000000000000000     <absolute>
 0000:00000000       ___safe_se_handler_table   0000000000000000     <absolute>
 0000:00000000       __arm64x_extra_rfe_table   0000000000000000     <absolute>
 0000:00000000       __arm64x_extra_rfe_table_size 0000000000000000     <absolute>
 0000:00000000       __arm64x_native_entrypoint 0000000000000000     <absolute>
 0000:00000000       __arm64x_redirection_metadata 0000000000000000     <absolute>
 0000:00000000       __arm64x_redirection_metadata_count 0000000000000000     <absolute>
 0000:00000000       __dynamic_value_reloc_table 0000000000000000     <absolute>
 0000:00000000       __enclave_config           0000000000000000     <absolute>
 0000:00000000       __guard_check_icall_a64n_fptr 0000000000000000     <absolute>
 0000:00000000       __guard_eh_cont_count      0000000000000000     <absolute>
 0000:00000000       __guard_eh_cont_table      0000000000000000     <absolute>
 0000:00000000       __guard_fids_count         0000000000000000     <absolute>
 0000:00000000       __guard_fids_table         0000000000000000     <absolute>
 0000:00000000       __guard_iat_count          0000000000000000     <absolute>
 0000:00000000       __guard_iat_table          0000000000000000     <absolute>
 0000:00000000       __guard_longjmp_count      0000000000000000     <absolute>
 0000:00000000       __guard_longjmp_table      0000000000000000     <absolute>
 0000:00000000       __hybrid_auxiliary_iat     0000000000000000     <absolute>
 0000:00000000       __hybrid_auxiliary_iat_copy 0000000000000000     <absolute>
 0000:00000000       __hybrid_code_map          0000000000000000     <absolute>
 0000:00000000       __hybrid_code_map_count    0000000000000000     <absolute>
 0000:00000000       __x64_code_ranges_to_entry_points 0000000000000000     <absolute>
 0000:00000000       __x64_code_ranges_to_entry_points_count 0000000000000000     <absolute>
 0000:00000100       __guard_flags              0000000000000100     <absolute>
 0000:00000000       __ImageBase                0000000180000000     <linker-defined>
 0001:00000000       ?SetEventNotificationMode@_jvmtiEnv@@QEAA?AW4jvmtiError@@W4jvmtiEventMode@@W4jvmtiEvent@@PEAV_jobject@@ZZ 0000000180001000 f i libNotifyFramePopStressTest.obj
 0001:0000000c       ?TranslateError@@YAPEBDW4jvmtiError@@@Z 000000018000100c f   libNotifyFramePopStressTest.obj
 0001:00000898       Agent_OnAttach             0000000180001898 f   libNotifyFramePopStressTest.obj
 0001:00000898       Agent_OnLoad               0000000180001898 f   libNotifyFramePopStressTest.obj
 0001:00000a18       JNI_OnLoad                 0000000180001a18 f   libNotifyFramePopStressTest.obj
 0001:00000a20       Java_NotifyFramePopStressTest_canGenerateFramePopEvents 0000000180001a20 f   libNotifyFramePopStressTest.obj
 0001:00000a2c       Java_NotifyFramePopStressTest_failed 0000000180001a2c f   libNotifyFramePopStressTest.obj
 0001:00000a34       Java_NotifyFramePopStressTest_getPopCount 0000000180001a34 f   libNotifyFramePopStressTest.obj
 0001:00000a3c       Java_NotifyFramePopStressTest_notifyFramePop 0000000180001a3c f   libNotifyFramePopStressTest.obj
 0001:00000bd8       Java_NotifyFramePopStressTest_resume 0000000180001bd8 f   libNotifyFramePopStressTest.obj
 0001:00000c0c       Java_NotifyFramePopStressTest_setFramePopNotificationMode 0000000180001c0c f   libNotifyFramePopStressTest.obj
 0001:00000c44       Java_NotifyFramePopStressTest_suspend 0000000180001c44 f   libNotifyFramePopStressTest.obj
 0001:00000c78       __local_stdio_printf_options 0000000180001c78 f i libNotifyFramePopStressTest.obj
 0001:00000c80       printf                     0000000180001c80 f i libNotifyFramePopStressTest.obj
 0001:00000dc8       _Init_thread_footer        0000000180001dc8 f   MSVCRT:thread_safe_statics.obj
 0001:00000e28       _Init_thread_header        0000000180001e28 f   MSVCRT:thread_safe_statics.obj
 0001:00000e90       _Init_thread_notify        0000000180001e90 f   MSVCRT:thread_safe_statics.obj
 0001:00000ed4       _Init_thread_wait          0000000180001ed4 f   MSVCRT:thread_safe_statics.obj
 0001:00000f38       __GSHandlerCheck           0000000180001f38 f   MSVCRT:gshandler.obj
 0001:00000f58       __GSHandlerCheckCommon     0000000180001f58 f   MSVCRT:gshandler.obj
 0001:00000fd0       __security_check_cookie    0000000180001fd0 f   MSVCRT:amdsecgs.obj
 0001:00001310       _DllMainCRTStartup         0000000180002310 f   MSVCRT:dll_dllmain.obj
 0001:00001350       __scrt_acquire_startup_lock 0000000180002350 f   MSVCRT:utility.obj
 0001:0000138c       __scrt_dllmain_after_initialize_c 000000018000238c f   MSVCRT:utility.obj
 0001:000013c0       __scrt_dllmain_before_initialize_c 00000001800023c0 f   MSVCRT:utility.obj
 0001:000013d8       __scrt_dllmain_crt_thread_attach 00000001800023d8 f   MSVCRT:utility.obj
 0001:00001400       __scrt_dllmain_crt_thread_detach 0000000180002400 f   MSVCRT:utility.obj
 0001:00001418       __scrt_dllmain_exception_filter 0000000180002418 f   MSVCRT:utility.obj
 0001:00001478       __scrt_dllmain_uninitialize_c 0000000180002478 f   MSVCRT:utility.obj
 0001:000014a8       __scrt_dllmain_uninitialize_critical 00000001800024a8 f   MSVCRT:utility.obj
 0001:000014bc       __scrt_initialize_crt      00000001800024bc f   MSVCRT:utility.obj
 0001:00001508       __scrt_initialize_onexit_tables 0000000180002508 f   MSVCRT:utility.obj
 0001:00001594       __scrt_is_nonwritable_in_current_image 0000000180002594 f   MSVCRT:utility.obj
 0001:0000162c       __scrt_release_startup_lock 000000018000262c f   MSVCRT:utility.obj
 0001:00001650       __scrt_uninitialize_crt    0000000180002650 f   MSVCRT:utility.obj
 0001:0000167c       _onexit                    000000018000267c f   MSVCRT:utility.obj
 0001:000016b8       atexit                     00000001800026b8 f   MSVCRT:utility.obj
 0001:000016d0       __crt_debugger_hook        00000001800026d0 f   MSVCRT:utility_desktop.obj
 0001:000016d8       __scrt_fastfail            00000001800026d8 f   MSVCRT:utility_desktop.obj
 0001:00001824       _guard_check_icall_nop     0000000180002824 f i MSVCRT:guard_support.obj
 0001:00001828       __raise_securityfailure    0000000180002828 f   MSVCRT:gs_report.obj
 0001:0000185c       __report_gsfailure         000000018000285c f   MSVCRT:gs_report.obj
 0001:000019a4       __security_init_cookie     00000001800029a4 f   MSVCRT:gs_support.obj
 0001:00001a50       DllMain                    0000000180002a50 f   MSVCRT:dll_dllmain_stub.obj
 0001:00001a74       ?__scrt_initialize_type_info@@YAXXZ 0000000180002a74 f   MSVCRT:tncleanup.obj
 0001:00001a84       ?__scrt_uninitialize_type_info@@YAXXZ 0000000180002a84 f   MSVCRT:tncleanup.obj
 0001:00001a90       __local_stdio_scanf_options 0000000180002a90 f i MSVCRT:default_local_stdio_options.obj
 0001:00001a98       __scrt_initialize_default_local_stdio_options 0000000180002a98 f   MSVCRT:default_local_stdio_options.obj
 0001:00001ab4       __scrt_get_dyn_tls_init_callback 0000000180002ab4 f   MSVCRT:dyn_tls_init.obj
 0001:00001abc       _RTC_Initialize            0000000180002abc f   MSVCRT:initsect.obj
 0001:00001af8       _RTC_Terminate             0000000180002af8 f   MSVCRT:initsect.obj
 0001:00001b34       __isa_available_init       0000000180002b34 f   MSVCRT:cpu_disp.obj
 0001:00001ce0       _get_startup_argv_mode     0000000180002ce0 f   MSVCRT:argv_mode.obj
 0001:00001ce8       __scrt_is_ucrt_dll_in_use  0000000180002ce8 f   MSVCRT:ucrt_detection.obj
 0001:00001d00       memset                     0000000180002d00 f   vcruntime:VCRUNTIME140.dll
 0001:00001d06       __C_specific_handler       0000000180002d06 f   vcruntime:VCRUNTIME140.dll
 0001:00001d0c       __std_type_info_destroy_list 0000000180002d0c f   vcruntime:VCRUNTIME140.dll
 0001:00001d12       strcmp                     0000000180002d12 f   ucrt:api-ms-win-crt-string-l1-1-0.dll
 0001:00001d18       strlen                     0000000180002d18 f   ucrt:api-ms-win-crt-string-l1-1-0.dll
 0001:00001d1e       _initterm                  0000000180002d1e f   ucrt:api-ms-win-crt-runtime-l1-1-0.dll
 0001:00001d24       _initterm_e                0000000180002d24 f   ucrt:api-ms-win-crt-runtime-l1-1-0.dll
 0001:00001d2a       _seh_filter_dll            0000000180002d2a f   ucrt:api-ms-win-crt-runtime-l1-1-0.dll
 0001:00001d30       _configure_narrow_argv     0000000180002d30 f   ucrt:api-ms-win-crt-runtime-l1-1-0.dll
 0001:00001d36       _initialize_narrow_environment 0000000180002d36 f   ucrt:api-ms-win-crt-runtime-l1-1-0.dll
 0001:00001d3c       _initialize_onexit_table   0000000180002d3c f   ucrt:api-ms-win-crt-runtime-l1-1-0.dll
 0001:00001d42       _register_onexit_function  0000000180002d42 f   ucrt:api-ms-win-crt-runtime-l1-1-0.dll
 0001:00001d48       _execute_onexit_table      0000000180002d48 f   ucrt:api-ms-win-crt-runtime-l1-1-0.dll
 0001:00001d4e       _crt_atexit                0000000180002d4e f   ucrt:api-ms-win-crt-runtime-l1-1-0.dll
 0001:00001d54       _cexit                     0000000180002d54 f   ucrt:api-ms-win-crt-runtime-l1-1-0.dll
 0001:00001d5c       __acrt_initialize          0000000180002d5c f   MSVCRT:ucrt_stubs.obj
 0001:00001d5c       __acrt_thread_attach       0000000180002d5c f   MSVCRT:ucrt_stubs.obj
 0001:00001d5c       __acrt_thread_detach       0000000180002d5c f   MSVCRT:ucrt_stubs.obj
 0001:00001d5c       __acrt_uninitialize        0000000180002d5c f   MSVCRT:ucrt_stubs.obj
 0001:00001d5c       __acrt_uninitialize_critical 0000000180002d5c f   MSVCRT:ucrt_stubs.obj
 0001:00001d5c       __scrt_stub_for_acrt_initialize 0000000180002d5c f   MSVCRT:ucrt_stubs.obj
 0001:00001d5c       __scrt_stub_for_acrt_thread_attach 0000000180002d5c f   MSVCRT:ucrt_stubs.obj
 0001:00001d5c       __scrt_stub_for_acrt_thread_detach 0000000180002d5c f   MSVCRT:ucrt_stubs.obj
 0001:00001d5c       __scrt_stub_for_acrt_uninitialize 0000000180002d5c f   MSVCRT:ucrt_stubs.obj
 0001:00001d5c       __scrt_stub_for_acrt_uninitialize_critical 0000000180002d5c f   MSVCRT:ucrt_stubs.obj
 0001:00001d5c       __vcrt_initialize          0000000180002d5c f   MSVCRT:ucrt_stubs.obj
 0001:00001d5c       __vcrt_thread_attach       0000000180002d5c f   MSVCRT:ucrt_stubs.obj
 0001:00001d5c       __vcrt_thread_detach       0000000180002d5c f   MSVCRT:ucrt_stubs.obj
 0001:00001d5c       __vcrt_uninitialize        0000000180002d5c f   MSVCRT:ucrt_stubs.obj
 0001:00001d5c       __vcrt_uninitialize_critical 0000000180002d5c f   MSVCRT:ucrt_stubs.obj
 0001:00001d60       __scrt_stub_for_is_c_termination_complete 0000000180002d60 f   MSVCRT:ucrt_stubs.obj
 0001:00001d60       _is_c_termination_complete 0000000180002d60 f   MSVCRT:ucrt_stubs.obj
 0001:00001d63       memcpy                     0000000180002d63 f   vcruntime:VCRUNTIME140.dll
 0001:00001d80       _guard_dispatch_icall_nop  0000000180002d80 f   MSVCRT:guard_dispatch.obj
 0001:00001da0       _guard_xfg_dispatch_icall_nop 0000000180002da0 f   MSVCRT:guard_xfg_dispatch.obj
 0002:00000000       __imp_CloseHandle          0000000180003000     kernel32:KERNEL32.dll
 0002:00000008       __imp_EnterCriticalSection 0000000180003008     kernel32:KERNEL32.dll
 0002:00000010       __imp_LeaveCriticalSection 0000000180003010     kernel32:KERNEL32.dll
 0002:00000018       __imp_InitializeCriticalSectionAndSpinCount 0000000180003018     kernel32:KERNEL32.dll
 0002:00000020       __imp_DeleteCriticalSection 0000000180003020     kernel32:KERNEL32.dll
 0002:00000028       __imp_SetEvent             0000000180003028     kernel32:KERNEL32.dll
 0002:00000030       __imp_ResetEvent           0000000180003030     kernel32:KERNEL32.dll
 0002:00000038       __imp_WaitForSingleObjectEx 0000000180003038     kernel32:KERNEL32.dll
 0002:00000040       __imp_CreateEventW         0000000180003040     kernel32:KERNEL32.dll
 0002:00000048       __imp_GetModuleHandleW     0000000180003048     kernel32:KERNEL32.dll
 0002:00000050       __imp_GetProcAddress       0000000180003050     kernel32:KERNEL32.dll
 0002:00000058       __imp_RtlCaptureContext    0000000180003058     kernel32:KERNEL32.dll
 0002:00000060       __imp_RtlLookupFunctionEntry 0000000180003060     kernel32:KERNEL32.dll
 0002:00000068       __imp_RtlVirtualUnwind     0000000180003068     kernel32:KERNEL32.dll
 0002:00000070       __imp_IsDebuggerPresent    0000000180003070     kernel32:KERNEL32.dll
 0002:00000078       __imp_UnhandledExceptionFilter 0000000180003078     kernel32:KERNEL32.dll
 0002:00000080       __imp_SetUnhandledExceptionFilter 0000000180003080     kernel32:KERNEL32.dll
 0002:00000088       __imp_IsProcessorFeaturePresent 0000000180003088     kernel32:KERNEL32.dll
 0002:00000090       __imp_GetCurrentProcess    0000000180003090     kernel32:KERNEL32.dll
 0002:00000098       __imp_TerminateProcess     0000000180003098     kernel32:KERNEL32.dll
 0002:000000a0       __imp_QueryPerformanceCounter 00000001800030a0     kernel32:KERNEL32.dll
 0002:000000a8       __imp_GetCurrentProcessId  00000001800030a8     kernel32:KERNEL32.dll
 0002:000000b0       __imp_GetCurrentThreadId   00000001800030b0     kernel32:KERNEL32.dll
 0002:000000b8       __imp_GetSystemTimeAsFileTime 00000001800030b8     kernel32:KERNEL32.dll
 0002:000000c0       __imp_DisableThreadLibraryCalls 00000001800030c0     kernel32:KERNEL32.dll
 0002:000000c8       __imp_InitializeSListHead  00000001800030c8     kernel32:KERNEL32.dll
 0002:000000d0       \177KERNEL32_NULL_THUNK_DATA 00000001800030d0     kernel32:KERNEL32.dll
 0002:000000d8       __imp_memset               00000001800030d8     vcruntime:VCRUNTIME140.dll
 0002:000000e0       __imp___C_specific_handler 00000001800030e0     vcruntime:VCRUNTIME140.dll
 0002:000000e8       __imp___std_type_info_destroy_list 00000001800030e8     vcruntime:VCRUNTIME140.dll
 0002:000000f0       __imp_memcpy               00000001800030f0     vcruntime:VCRUNTIME140.dll
 0002:000000f8       \177VCRUNTIME140_NULL_THUNK_DATA 00000001800030f8     vcruntime:VCRUNTIME140.dll
 0002:00000100       __imp__initialize_narrow_environment 0000000180003100     ucrt:api-ms-win-crt-runtime-l1-1-0.dll
 0002:00000108       __imp__cexit               0000000180003108     ucrt:api-ms-win-crt-runtime-l1-1-0.dll
 0002:00000110       __imp__crt_atexit          0000000180003110     ucrt:api-ms-win-crt-runtime-l1-1-0.dll
 0002:00000118       __imp__execute_onexit_table 0000000180003118     ucrt:api-ms-win-crt-runtime-l1-1-0.dll
 0002:00000120       __imp__register_onexit_function 0000000180003120     ucrt:api-ms-win-crt-runtime-l1-1-0.dll
 0002:00000128       __imp_abort                0000000180003128     ucrt:api-ms-win-crt-runtime-l1-1-0.dll
 0002:00000130       __imp__initterm            0000000180003130     ucrt:api-ms-win-crt-runtime-l1-1-0.dll
 0002:00000138       __imp__initterm_e          0000000180003138     ucrt:api-ms-win-crt-runtime-l1-1-0.dll
 0002:00000140       __imp__seh_filter_dll      0000000180003140     ucrt:api-ms-win-crt-runtime-l1-1-0.dll
 0002:00000148       __imp__initialize_onexit_table 0000000180003148     ucrt:api-ms-win-crt-runtime-l1-1-0.dll
 0002:00000150       __imp__configure_narrow_argv 0000000180003150     ucrt:api-ms-win-crt-runtime-l1-1-0.dll
 0002:00000158       \177api-ms-win-crt-runtime-l1-1-0_NULL_THUNK_DATA 0000000180003158     ucrt:api-ms-win-crt-runtime-l1-1-0.dll
 0002:00000160       __imp___acrt_iob_func      0000000180003160     ucrt:api-ms-win-crt-stdio-l1-1-0.dll
 0002:00000168       __imp___stdio_common_vfprintf 0000000180003168     ucrt:api-ms-win-crt-stdio-l1-1-0.dll
 0002:00000170       __imp_fflush               0000000180003170     ucrt:api-ms-win-crt-stdio-l1-1-0.dll
 0002:00000178       \177api-ms-win-crt-stdio-l1-1-0_NULL_THUNK_DATA 0000000180003178     ucrt:api-ms-win-crt-stdio-l1-1-0.dll
 0002:00000180       __imp_strlen               0000000180003180     ucrt:api-ms-win-crt-string-l1-1-0.dll
 0002:00000188       __imp_strncpy              0000000180003188     ucrt:api-ms-win-crt-string-l1-1-0.dll
 0002:00000190       __imp_strcmp               0000000180003190     ucrt:api-ms-win-crt-string-l1-1-0.dll
 0002:00000198       \177api-ms-win-crt-string-l1-1-0_NULL_THUNK_DATA 0000000180003198     ucrt:api-ms-win-crt-string-l1-1-0.dll
 0002:000001a0       __guard_check_icall_fptr   00000001800031a0     MSVCRT:guard_support.obj
 0002:000001a8       __guard_xfg_check_icall_fptr 00000001800031a8     MSVCRT:guard_support.obj
 0002:000001b0       __guard_dispatch_icall_fptr 00000001800031b0     MSVCRT:guard_support.obj
 0002:000001b8       __guard_xfg_dispatch_icall_fptr 00000001800031b8     MSVCRT:guard_support.obj
 0002:000001c0       __guard_xfg_table_dispatch_icall_fptr 00000001800031c0     MSVCRT:guard_support.obj
 0002:000001c8       __castguard_check_failure_os_handled_fptr 00000001800031c8     MSVCRT:guard_support.obj
 0002:000001d0       __guard_memcpy_fptr        00000001800031d0     vcruntime:softmemtag.obj
 0002:000001d8       __xc_a                     00000001800031d8     MSVCRT:initializers.obj
 0002:000001e0       __xc_z                     00000001800031e0     MSVCRT:initializers.obj
 0002:000001e8       __xi_a                     00000001800031e8     MSVCRT:initializers.obj
 0002:000001f8       __xi_z                     00000001800031f8     MSVCRT:initializers.obj
 0002:00000200       __xl_a                     0000000180003200     MSVCRT:tlssup.obj
 0002:00000208       __xl_z                     0000000180003208     MSVCRT:tlssup.obj
 0002:00000210       __xp_a                     0000000180003210     MSVCRT:initializers.obj
 0002:00000218       __xp_z                     0000000180003218     MSVCRT:initializers.obj
 0002:00000220       __xt_a                     0000000180003220     MSVCRT:initializers.obj
 0002:00000228       __xt_z                     0000000180003228     MSVCRT:initializers.obj
 0002:00000230       ??_C@_0DO@CIJFOGIH@check_jvmti_error?3?5JVMTI?5functi@ 0000000180003230     libNotifyFramePopStressTest.obj
 0002:00000270       ??_C@_0DM@KLJPMIDM@check_jvmti_status?3?5JVMTI?5funct@ 0000000180003270     libNotifyFramePopStressTest.obj
 0002:000002b0       ??_C@_0CL@MEELKAEL@deallocate?3?5error?5in?5JVMTI?5Deal@ 00000001800032b0     libNotifyFramePopStressTest.obj
 0002:000002e0       ??_C@_0DO@CNKPCOHC@get_method_class_name?3?5error?5in@ 00000001800032e0     libNotifyFramePopStressTest.obj
 0002:00000320       ??_C@_0DI@ODOBMANA@get_method_class_name?3?5error?5in@ 0000000180003320     libNotifyFramePopStressTest.obj
 0002:00000358       ??_C@_0CP@IBPBEBM@get_method_class_name?3?5error?5in@ 0000000180003358     libNotifyFramePopStressTest.obj
 0002:00000388       ??_C@_0CL@BDMIAND@print_method?3?5error?5in?5JVMTI?5Ge@ 0000000180003388     libNotifyFramePopStressTest.obj
 0002:000003b8       ??_C@_0P@GFDDDNG@?$CF2d?3?5?$CFs?3?5?$CFs?$CFs?6@ 00000001800033b8     libNotifyFramePopStressTest.obj
 0002:000003c8       ??_C@_01EEMJAFIK@?6@       00000001800033c8     libNotifyFramePopStressTest.obj
 0002:000003d0       ??_C@_0DB@CBIFKKAL@notifyFramePop?3?5Failed?5in?5JVMTI@ 00000001800033d0     libNotifyFramePopStressTest.obj
 0002:00000408       ??_C@_0BB@NEONAMMP@?$DMUnnamed?5thread?$DO@ 0000000180003408     libNotifyFramePopStressTest.obj
 0002:00000420       ??_C@_0DD@PEIMAGBL@get_thread_name?3?5error?5in?5JVMTI@ 0000000180003420     libNotifyFramePopStressTest.obj
 0002:00000458       ??_C@_0DD@GMADJBLO@get_method_name?3?5error?5in?5JVMTI@ 0000000180003458     libNotifyFramePopStressTest.obj
 0002:00000490       ??_C@_0DA@DGJBBBMN@print_stack_trace?3?5error?5in?5JVM@ 0000000180003490     libNotifyFramePopStressTest.obj
 0002:000004c0       ??_C@_0DC@EJGPEKOE@JVMTI?5Stack?5Trace?5for?5thread?5?$CFs@ 00000001800034c0     libNotifyFramePopStressTest.obj
 0002:000004f8       ??_C@_0BN@DPBGGNAC@error?5in?5JVMTI?5SuspendThread@ 00000001800034f8     libNotifyFramePopStressTest.obj
 0002:00000518       ??_C@_0BM@HOJKOFIM@error?5in?5JVMTI?5ResumeThread@ 0000000180003518     libNotifyFramePopStressTest.obj
 0002:00000538       ??_C@_0BB@JCNMKLLK@JVMTI_ERROR_NONE@ 0000000180003538     libNotifyFramePopStressTest.obj
 0002:00000550       ??_C@_0BL@LDIMKLPH@JVMTI_ERROR_INVALID_THREAD@ 0000000180003550     libNotifyFramePopStressTest.obj
 0002:00000570       ??_C@_0CB@PJFPAIKJ@JVMTI_ERROR_INVALID_THREAD_GROU@ 0000000180003570     libNotifyFramePopStressTest.obj
 0002:00000598       ??_C@_0BN@LLMKHMNF@JVMTI_ERROR_INVALID_PRIORITY@ 0000000180003598     libNotifyFramePopStressTest.obj
 0002:000005b8       ??_C@_0CB@MBOFKAGB@JVMTI_ERROR_THREAD_NOT_SUSPENDE@ 00000001800035b8     libNotifyFramePopStressTest.obj
 0002:000005e0       ??_C@_0BN@FABOLPBI@JVMTI_ERROR_THREAD_SUSPENDED@ 00000001800035e0     libNotifyFramePopStressTest.obj
 0002:00000600       ??_C@_0BN@FDGNOBJM@JVMTI_ERROR_THREAD_NOT_ALIVE@ 0000000180003600     libNotifyFramePopStressTest.obj
 0002:00000620       ??_C@_0BL@GOBIFKNJ@JVMTI_ERROR_INVALID_OBJECT@ 0000000180003620     libNotifyFramePopStressTest.obj
 0002:00000640       ??_C@_0BK@FCMAJPPC@JVMTI_ERROR_INVALID_CLASS@ 0000000180003640     libNotifyFramePopStressTest.obj
 0002:00000660       ??_C@_0BP@IKLLBKEB@JVMTI_ERROR_CLASS_NOT_PREPARED@ 0000000180003660     libNotifyFramePopStressTest.obj
 0002:00000680       ??_C@_0BN@KLPPLKG@JVMTI_ERROR_INVALID_METHODID@ 0000000180003680     libNotifyFramePopStressTest.obj
 0002:000006a0       ??_C@_0BN@BCEKOKND@JVMTI_ERROR_INVALID_LOCATION@ 00000001800036a0     libNotifyFramePopStressTest.obj
 0002:000006c0       ??_C@_0BM@DFDGPME@JVMTI_ERROR_INVALID_FIELDID@ 00000001800036c0     libNotifyFramePopStressTest.obj
 0002:000006e0       ??_C@_0BL@NELIEPEC@JVMTI_ERROR_NO_MORE_FRAMES@ 00000001800036e0     libNotifyFramePopStressTest.obj
 0002:00000700       ??_C@_0BJ@BDBECFDM@JVMTI_ERROR_OPAQUE_FRAME@ 0000000180003700     libNotifyFramePopStressTest.obj
 0002:00000720       ??_C@_0BK@MIIFNLOB@JVMTI_ERROR_TYPE_MISMATCH@ 0000000180003720     libNotifyFramePopStressTest.obj
 0002:00000740       ??_C@_0BJ@HPCAOILC@JVMTI_ERROR_INVALID_SLOT@ 0000000180003740     libNotifyFramePopStressTest.obj
 0002:00000760       ??_C@_0BG@CHILOPNI@JVMTI_ERROR_DUPLICATE@ 0000000180003760     libNotifyFramePopStressTest.obj
 0002:00000778       ??_C@_0BG@DIEMLHKM@JVMTI_ERROR_NOT_FOUND@ 0000000180003778     libNotifyFramePopStressTest.obj
 0002:00000790       ??_C@_0BM@NHMCKHOB@JVMTI_ERROR_INVALID_MONITOR@ 0000000180003790     libNotifyFramePopStressTest.obj
 0002:000007b0       ??_C@_0BO@PPEDAJGL@JVMTI_ERROR_NOT_MONITOR_OWNER@ 00000001800037b0     libNotifyFramePopStressTest.obj
 0002:000007d0       ??_C@_0BG@FCAIPEID@JVMTI_ERROR_INTERRUPT@ 00000001800037d0     libNotifyFramePopStressTest.obj
 0002:000007e8       ??_C@_0CB@EGDBNKOI@JVMTI_ERROR_INVALID_CLASS_FORMA@ 00000001800037e8     libNotifyFramePopStressTest.obj
 0002:00000810       ??_C@_0CG@DGKOGIAL@JVMTI_ERROR_CIRCULAR_CLASS_DEFI@ 0000000180003810     libNotifyFramePopStressTest.obj
 0002:00000838       ??_C@_0BP@ICEALPKC@JVMTI_ERROR_FAILS_VERIFICATION@ 0000000180003838     libNotifyFramePopStressTest.obj
 0002:00000858       ??_C@_0DC@JDACLMIO@JVMTI_ERROR_UNSUPPORTED_REDEFIN@ 0000000180003858     libNotifyFramePopStressTest.obj
 0002:00000890       ??_C@_0DE@GKDKNOMJ@JVMTI_ERROR_UNSUPPORTED_REDEFIN@ 0000000180003890     libNotifyFramePopStressTest.obj
 0002:000008c8       ??_C@_0BO@LAFKIOG@JVMTI_ERROR_INVALID_TYPESTATE@ 00000001800038c8     libNotifyFramePopStressTest.obj
 0002:000008e8       ??_C@_0DH@INDGCLLB@JVMTI_ERROR_UNSUPPORTED_REDEFIN@ 00000001800038e8     libNotifyFramePopStressTest.obj
 0002:00000920       ??_C@_0DE@NHEOMMGI@JVMTI_ERROR_UNSUPPORTED_REDEFIN@ 0000000180003920     libNotifyFramePopStressTest.obj
 0002:00000958       ??_C@_0CA@EKPNJOEP@JVMTI_ERROR_UNSUPPORTED_VERSION@ 0000000180003958     libNotifyFramePopStressTest.obj
 0002:00000978       ??_C@_0BN@OFFMAHHL@JVMTI_ERROR_NAMES_DONT_MATCH@ 0000000180003978     libNotifyFramePopStressTest.obj
 0002:00000998       ??_C@_0DN@HHBBLAKE@JVMTI_ERROR_UNSUPPORTED_REDEFIN@ 0000000180003998     libNotifyFramePopStressTest.obj
 0002:000009d8       ??_C@_0DO@HMBGBGNA@JVMTI_ERROR_UNSUPPORTED_REDEFIN@ 00000001800039d8     libNotifyFramePopStressTest.obj
 0002:00000a18       ??_C@_0BP@PBECGKHJ@JVMTI_ERROR_UNMODIFIABLE_CLASS@ 0000000180003a18     libNotifyFramePopStressTest.obj
 0002:00000a38       ??_C@_0BK@CANILEHF@JVMTI_ERROR_NOT_AVAILABLE@ 0000000180003a38     libNotifyFramePopStressTest.obj
 0002:00000a58       ??_C@_0CE@INJKMEFK@JVMTI_ERROR_MUST_POSSESS_CAPABI@ 0000000180003a58     libNotifyFramePopStressTest.obj
 0002:00000a80       ??_C@_0BJ@LBFPFPDM@JVMTI_ERROR_NULL_POINTER@ 0000000180003a80     libNotifyFramePopStressTest.obj
 0002:00000aa0       ??_C@_0BP@CHJPNNEM@JVMTI_ERROR_ABSENT_INFORMATION@ 0000000180003aa0     libNotifyFramePopStressTest.obj
 0002:00000ac0       ??_C@_0BP@OMFMNLC@JVMTI_ERROR_INVALID_EVENT_TYPE@ 0000000180003ac0     libNotifyFramePopStressTest.obj
 0002:00000ae0       ??_C@_0BN@BIBNPHHO@JVMTI_ERROR_ILLEGAL_ARGUMENT@ 0000000180003ae0     libNotifyFramePopStressTest.obj
 0002:00000b00       ??_C@_0BK@KKNDHDCE@JVMTI_ERROR_NATIVE_METHOD@ 0000000180003b00     libNotifyFramePopStressTest.obj
 0002:00000b20       ??_C@_0BK@PMKCFHAE@JVMTI_ERROR_OUT_OF_MEMORY@ 0000000180003b20     libNotifyFramePopStressTest.obj
 0002:00000b40       ??_C@_0BK@NNJBDMNB@JVMTI_ERROR_ACCESS_DENIED@ 0000000180003b40     libNotifyFramePopStressTest.obj
 0002:00000b60       ??_C@_0BI@GHECLMNC@JVMTI_ERROR_WRONG_PHASE@ 0000000180003b60     libNotifyFramePopStressTest.obj
 0002:00000b78       ??_C@_0BF@OLIHJOII@JVMTI_ERROR_INTERNAL@ 0000000180003b78     libNotifyFramePopStressTest.obj
 0002:00000b90       ??_C@_0BO@EOHGKJHI@JVMTI_ERROR_UNATTACHED_THREAD@ 0000000180003b90     libNotifyFramePopStressTest.obj
 0002:00000bb0       ??_C@_0CA@LKHFDACL@JVMTI_ERROR_INVALID_ENVIRONMENT@ 0000000180003bb0     libNotifyFramePopStressTest.obj
 0002:00000bd0       ??_C@_0BA@MMFHLOKK@?$DMunknown?5error?$DO@ 0000000180003bd0     libNotifyFramePopStressTest.obj
 0002:00000be0       ??_C@_0FC@DIHHIAJG@jvmti_common?5set_event_notifica@ 0000000180003be0     libNotifyFramePopStressTest.obj
 0002:00000c38       ??_C@_0DC@LADLMCBP@FramePop?3?5Failed?5in?5JVMTI?5GetMe@ 0000000180003c38     libNotifyFramePopStressTest.obj
 0002:00000c70       ??_C@_0CM@JAIMFDJE@FramePop?3?5Failed?5in?5JVMTI?5GetCl@ 0000000180003c70     libNotifyFramePopStressTest.obj
 0002:00000ca0       ??_C@_0CH@CDFMOFDK@FramePop?$CI?$CFd?$CJ?5event?5from?5method?3@ 0000000180003ca0     libNotifyFramePopStressTest.obj
 0002:00000cc8       ??_C@_04GHJNJNPO@main@     0000000180003cc8     libNotifyFramePopStressTest.obj
 0002:00000cd0       ??_C@_0EA@HJKKGEK@ERROR?3?5FramePop?5event?5is?5for?5wr@ 0000000180003cd0     libNotifyFramePopStressTest.obj
 0002:00000d10       ??_C@_0CJ@LOGGFPCM@GetEnv?$CIJVMTI_VERSION_9?$CJ?5failed?5@ 0000000180003d10     libNotifyFramePopStressTest.obj
 0002:00000d40       ??_C@_0CH@KCBABMIN@Agent?3?5GetPotentialCapabilities@ 0000000180003d40     libNotifyFramePopStressTest.obj
 0002:00000d68       ??_C@_0BO@BBCJDFNJ@Agent?3?5AddCapabilities?5failed@ 0000000180003d68     libNotifyFramePopStressTest.obj
 0002:00000d88       ??_C@_0BO@KACPDBIP@Agent?3?5GetCapabilities?5failed@ 0000000180003d88     libNotifyFramePopStressTest.obj
 0002:00000da8       ??_C@_0CA@OPCEMBMO@Agent?3?5SetEventCallbacks?5failed@ 0000000180003da8     libNotifyFramePopStressTest.obj
 0002:00000dc8       ??_C@_0CP@FIJCDEEJ@notifyFramePop?3?5Failed?5in?5JVMTI@ 0000000180003dc8     libNotifyFramePopStressTest.obj
 0002:00000e00       ??_C@_0EF@FOOMGKCK@?6notifyFramePop?3?5requested?5Fram@ 0000000180003e00     libNotifyFramePopStressTest.obj
 0002:00000e48       ??_C@_0CJ@CMKNLDJL@notifyFramePop?5not?5counting?5mai@ 0000000180003e48     libNotifyFramePopStressTest.obj
 0002:00000e80       ??_C@_1EC@JIJBPKFM@?$AAa?$AAp?$AAi?$AA?9?$AAm?$AAs?$AA?9?$AAw?$AAi?$AAn?$AA?9?$AAc?$AAo?$AAr?$AAe@ 0000000180003e80     MSVCRT:thread_safe_statics.obj
 0002:00000ec8       ??_C@_1BK@MGMFAEKH@?$AAk?$AAe?$AAr?$AAn?$AAe?$AAl?$AA3?$AA2?$AA?4?$AAd?$AAl?$AAl@ 0000000180003ec8     MSVCRT:thread_safe_statics.obj
 0002:00000ee8       ??_C@_0BJ@JEBJOJFJ@SleepConditionVariableCS@ 0000000180003ee8     MSVCRT:thread_safe_statics.obj
 0002:00000f08       ??_C@_0BJ@PGPPEPCC@WakeAllConditionVariable@ 0000000180003f08     MSVCRT:thread_safe_statics.obj
 0002:00000f28       _pDefaultRawDllMain        0000000180003f28     MSVCRT:dll_dllmain.obj
 0002:00000f28       _pRawDllMain               0000000180003f28     MSVCRT:dll_dllmain.obj
 0002:00000f30       __xmm@ffffffffffffffffffffffffffffffff 0000000180003f30     MSVCRT:utility.obj
 0002:00000f50       _load_config_used          0000000180003f50     MSVCRT:loadcfg.obj
 0002:00001100       _tls_used                  0000000180004100     MSVCRT:tlssup.obj
 0002:00001128       __volatile_metadata        0000000180004128     <linker-defined>
 0002:000014e0       __rtc_iaa                  00000001800044e0     MSVCRT:initsect.obj
 0002:000014e8       __rtc_izz                  00000001800044e8     MSVCRT:initsect.obj
 0002:000014f0       __rtc_taa                  00000001800044f0     MSVCRT:initsect.obj
 0002:000014f8       __rtc_tzz                  00000001800044f8     MSVCRT:initsect.obj
 0002:00001500       _tls_start                 0000000180004500     MSVCRT:tlssup.obj
 0002:00001504       _Init_thread_epoch         0000000180004504     MSVCRT:thread_safe_statics.obj
 0002:00001508       _tls_end                   0000000180004508     MSVCRT:tlssup.obj
 0002:0000191c       __IMPORT_DESCRIPTOR_KERNEL32 000000018000491c     kernel32:KERNEL32.dll
 0002:00001930       __IMPORT_DESCRIPTOR_VCRUNTIME140 0000000180004930     vcruntime:VCRUNTIME140.dll
 0002:00001944       __IMPORT_DESCRIPTOR_api-ms-win-crt-stdio-l1-1-0 0000000180004944     ucrt:api-ms-win-crt-stdio-l1-1-0.dll
 0002:00001958       __IMPORT_DESCRIPTOR_api-ms-win-crt-string-l1-1-0 0000000180004958     ucrt:api-ms-win-crt-string-l1-1-0.dll
 0002:0000196c       __IMPORT_DESCRIPTOR_api-ms-win-crt-runtime-l1-1-0 000000018000496c     ucrt:api-ms-win-crt-runtime-l1-1-0.dll
 0002:00001980       __NULL_IMPORT_DESCRIPTOR   0000000180004980     kernel32:KERNEL32.dll
 0003:00000008       _Init_global_epoch         0000000180005008     MSVCRT:thread_safe_statics.obj
 0003:00000010       __security_cookie          0000000180005010     MSVCRT:gs_cookie.obj
 0003:00000018       __security_cookie_complement 0000000180005018     MSVCRT:gs_cookie.obj
 0003:00000020       __scrt_native_dllmain_reason 0000000180005020     MSVCRT:utility.obj
 0003:00000028       __isa_available            0000000180005028     MSVCRT:cpu_disp.obj
 0003:0000002c       __isa_enabled              000000018000502c     MSVCRT:cpu_disp.obj
 0003:00000030       __memset_fast_string_threshold 0000000180005030     MSVCRT:cpu_disp.obj
 0003:00000038       __memset_nt_threshold      0000000180005038     MSVCRT:cpu_disp.obj
 0003:00000040       __scrt_ucrt_dll_is_in_use  0000000180005040     MSVCRT:ucrt_stubs.obj
 0003:00000050       ?_OptionsStorage@?1??__local_stdio_printf_options@@9@4_KA 0000000180005050     libNotifyFramePopStressTest.obj
 0003:00000218       _tls_index                 0000000180005218     MSVCRT:tlssup.obj
 0003:00000220       __scrt_current_native_startup_state 0000000180005220     MSVCRT:utility.obj
 0003:00000228       __scrt_native_startup_lock 0000000180005228     MSVCRT:utility.obj
 0003:00000268       __scrt_debugger_hook_flag  0000000180005268     MSVCRT:utility_desktop.obj
 0003:000007e0       ?__type_info_root_node@@3U__type_info_node@@A 00000001800057e0     MSVCRT:tncleanup.obj
 0003:000007f0       ?_OptionsStorage@?1??__local_stdio_scanf_options@@9@4_KA 00000001800057f0     MSVCRT:default_local_stdio_options.obj
 0003:000007f8       __favor                    00000001800057f8     MSVCRT:cpu_disp.obj
 0003:00000800       __dyn_tls_init_callback    0000000180005800     <common>

 entry point at        0001:00001310

 Static symbols

 0000:ffff8000       .debug$S                   0000000180000000     NotifyFramePopStressTest.exp
 0000:ffff8000       .debug$S                   0000000180000000     vcruntime:VCRUNTIME140.dll
 0000:ffff8000       .debug$S                   0000000180000000     vcruntime:VCRUNTIME140.dll
 0000:ffff8000       .debug$S                   0000000180000000     vcruntime:VCRUNTIME140.dll
 0000:ffff8000       .debug$S                   0000000180000000     vcruntime:VCRUNTIME140.dll
 0000:ffff8000       .debug$S                   0000000180000000     vcruntime:VCRUNTIME140.dll
 0000:ffff8000       .debug$S                   0000000180000000     vcruntime:VCRUNTIME140.dll
 0000:ffff8000       .debug$S                   0000000180000000     ucrt:api-ms-win-crt-runtime-l1-1-0.dll
 0000:ffff8000       .debug$S                   0000000180000000     ucrt:api-ms-win-crt-runtime-l1-1-0.dll
 0000:ffff8000       .debug$S                   0000000180000000     ucrt:api-ms-win-crt-runtime-l1-1-0.dll
 0000:ffff8000       .debug$S                   0000000180000000     ucrt:api-ms-win-crt-runtime-l1-1-0.dll
 0000:ffff8000       .debug$S                   0000000180000000     ucrt:api-ms-win-crt-runtime-l1-1-0.dll
 0000:ffff8000       .debug$S                   0000000180000000     ucrt:api-ms-win-crt-runtime-l1-1-0.dll
 0000:ffff8000       .debug$S                   0000000180000000     ucrt:api-ms-win-crt-runtime-l1-1-0.dll
 0000:ffff8000       .debug$S                   0000000180000000     ucrt:api-ms-win-crt-runtime-l1-1-0.dll
 0000:ffff8000       .debug$S                   0000000180000000     ucrt:api-ms-win-crt-runtime-l1-1-0.dll
 0000:ffff8000       .debug$S                   0000000180000000     ucrt:api-ms-win-crt-runtime-l1-1-0.dll
 0000:ffff8000       .debug$S                   0000000180000000     ucrt:api-ms-win-crt-runtime-l1-1-0.dll
 0000:ffff8000       .debug$S                   0000000180000000     ucrt:api-ms-win-crt-runtime-l1-1-0.dll
 0000:ffff8000       .debug$S                   0000000180000000     ucrt:api-ms-win-crt-runtime-l1-1-0.dll
 0000:ffff8000       .debug$S                   0000000180000000     ucrt:api-ms-win-crt-stdio-l1-1-0.dll
 0000:ffff8000       .debug$S                   0000000180000000     ucrt:api-ms-win-crt-stdio-l1-1-0.dll
 0000:ffff8000       .debug$S                   0000000180000000     ucrt:api-ms-win-crt-stdio-l1-1-0.dll
 0000:ffff8000       .debug$S                   0000000180000000     ucrt:api-ms-win-crt-string-l1-1-0.dll
 0000:ffff8000       .debug$S                   0000000180000000     ucrt:api-ms-win-crt-string-l1-1-0.dll
 0000:ffff8000       .debug$S                   0000000180000000     ucrt:api-ms-win-crt-string-l1-1-0.dll
 0000:ffff8000       .debug$S                   0000000180000000     ucrt:api-ms-win-crt-string-l1-1-0.dll
 0000:ffff8000       .debug$S                   0000000180000000     ucrt:api-ms-win-crt-string-l1-1-0.dll
 0000:ffff8000       .debug$S                   0000000180000000     kernel32:KERNEL32.dll
 0000:ffff8000       .debug$S                   0000000180000000     kernel32:KERNEL32.dll
 0000:ffff8000       .debug$S                   0000000180000000     kernel32:KERNEL32.dll
 0000:ffff8000       .debug$S                   0000000180000000     kernel32:KERNEL32.dll
 0000:ffff8000       .debug$S                   0000000180000000     kernel32:KERNEL32.dll
 0000:ffff8000       .debug$S                   0000000180000000     kernel32:KERNEL32.dll
 0000:ffff8000       .debug$S                   0000000180000000     kernel32:KERNEL32.dll
 0000:ffff8000       .debug$S                   0000000180000000     kernel32:KERNEL32.dll
 0000:ffff8000       .debug$S                   0000000180000000     kernel32:KERNEL32.dll
 0000:ffff8000       .debug$S                   0000000180000000     kernel32:KERNEL32.dll
 0000:ffff8000       .debug$S                   0000000180000000     kernel32:KERNEL32.dll
 0000:ffff8000       .debug$S                   0000000180000000     kernel32:KERNEL32.dll
 0000:ffff8000       .debug$S                   0000000180000000     kernel32:KERNEL32.dll
 0000:ffff8000       .debug$S                   0000000180000000     kernel32:KERNEL32.dll
 0000:ffff8000       .debug$S                   0000000180000000     kernel32:KERNEL32.dll
 0000:ffff8000       .debug$S                   0000000180000000     kernel32:KERNEL32.dll
 0000:ffff8000       .debug$S                   0000000180000000     kernel32:KERNEL32.dll
 0000:ffff8000       .debug$S                   0000000180000000     kernel32:KERNEL32.dll
 0000:ffff8000       .debug$S                   0000000180000000     kernel32:KERNEL32.dll
 0000:ffff8000       .debug$S                   0000000180000000     kernel32:KERNEL32.dll
 0000:ffff8000       .debug$S                   0000000180000000     kernel32:KERNEL32.dll
 0000:ffff8000       .debug$S                   0000000180000000     kernel32:KERNEL32.dll
 0000:ffff8000       .debug$S                   0000000180000000     kernel32:KERNEL32.dll
 0000:ffff8000       .debug$S                   0000000180000000     kernel32:KERNEL32.dll
 0000:ffff8000       .debug$S                   0000000180000000     kernel32:KERNEL32.dll
 0000:ffff8000       .debug$S                   0000000180000000     kernel32:KERNEL32.dll
 0000:ffff8000       .debug$S                   0000000180000000     kernel32:KERNEL32.dll
 0000:ffff8000       .debug$S                   0000000180000000     kernel32:KERNEL32.dll
 0001:000002c4       ?check_jvmti_error@@YAXW4jvmtiError@@PEBD@Z 00000001800012c4 f   libNotifyFramePopStressTest.obj
 0001:00000310       ?check_jvmti_status@@YAXPEAUJNIEnv_@@W4jvmtiError@@PEBD@Z 0000000180001310 f   libNotifyFramePopStressTest.obj
 0001:00000378       ?deallocate@@YAXPEAU_jvmtiEnv@@PEAUJNIEnv_@@PEAX@Z 0000000180001378 f   libNotifyFramePopStressTest.obj
 0001:000003a8       ?print_stack_trace@@YAXPEAU_jvmtiEnv@@PEAUJNIEnv_@@PEAV_jobject@@@Z 00000001800013a8 f   libNotifyFramePopStressTest.obj
 0001:00000778       Agent_Initialize           0000000180001778 f   libNotifyFramePopStressTest.obj
 0001:000008a0       FramePop                   00000001800018a0 f   libNotifyFramePopStressTest.obj
 0001:00000cd0       ?__scrt_initialize_thread_safe_statics@@YAHXZ 0000000180001cd0 f   MSVCRT:thread_safe_statics.obj
 0001:00000da0       ?__scrt_uninitialize_thread_safe_statics@@YAXXZ 0000000180001da0 f   MSVCRT:thread_safe_statics.obj
 0001:00000fc0       $$000000                   0000000180001fc0     MSVCRT:amdsecgs.obj
 0001:00000ff0       ?dllmain_crt_dispatch@@YAHQEAUHINSTANCE__@@KQEAX@Z 0000000180001ff0 f   MSVCRT:dll_dllmain.obj
 0001:00001040       ?dllmain_crt_process_attach@@YAHQEAUHINSTANCE__@@QEAX@Z 0000000180002040 f   MSVCRT:dll_dllmain.obj
 0001:00001158       ?dllmain_crt_process_detach@@YAH_N@Z 0000000180002158 f   MSVCRT:dll_dllmain.obj
 0001:000011dc       ?dllmain_dispatch@@YAHQEAUHINSTANCE__@@KQEAX@Z 00000001800021dc f   MSVCRT:dll_dllmain.obj
 0001:00001930       capture_previous_context   0000000180002930 f   MSVCRT:gs_report.obj
 0001:00001d70       $$000000                   0000000180002d70     MSVCRT:guard_dispatch.obj
 0001:00001d90       $$000000                   0000000180002d90     MSVCRT:guard_xfg_dispatch.obj
 0001:00001da6       ?fin$0@?0??dllmain_crt_process_attach@@YAHQEAUHINSTANCE__@@QEAX@Z@4HA 0000000180002da6 f   MSVCRT:dll_dllmain.obj
 0001:00001dbd       ?fin$0@?0??dllmain_crt_process_detach@@YAH_N@Z@4HA 0000000180002dbd f   MSVCRT:dll_dllmain.obj
 0001:00001dd6       ?fin$1@?0??dllmain_crt_process_detach@@YAH_N@Z@4HA 0000000180002dd6 f   MSVCRT:dll_dllmain.obj
 0001:00001dea       ?filt$0@?0??dllmain_dispatch@@YAHQEAUHINSTANCE__@@KQEAX@Z@4HA 0000000180002dea f   MSVCRT:dll_dllmain.obj
 0001:00001e20       __scrt_is_nonwritable_in_current_image$filt$0 0000000180002e20 f   MSVCRT:utility.obj
 0002:000001f0       ?__scrt_initialize_tss_var@@3P6AHXZEA 00000001800031f0     MSVCRT:thread_safe_statics.obj
 0002:00000f40       GS_ExceptionPointers       0000000180003f40     MSVCRT:gs_report.obj
 0002:00001510       $unwind$printf             0000000180004510     libNotifyFramePopStressTest.obj
 0002:0000151c       $unwind$?check_jvmti_error@@YAXW4jvmtiError@@PEBD@Z 000000018000451c     libNotifyFramePopStressTest.obj
 0002:00001528       $unwind$?check_jvmti_status@@YAXPEAUJNIEnv_@@W4jvmtiError@@PEBD@Z 0000000180004528     libNotifyFramePopStressTest.obj
 0002:00001538       $unwind$?deallocate@@YAXPEAU_jvmtiEnv@@PEAUJNIEnv_@@PEAX@Z 0000000180004538     libNotifyFramePopStressTest.obj
 0002:00001538       $unwind$Java_NotifyFramePopStressTest_resume 0000000180004538     libNotifyFramePopStressTest.obj
 0002:00001538       $unwind$Java_NotifyFramePopStressTest_setFramePopNotificationMode 0000000180004538     libNotifyFramePopStressTest.obj
 0002:00001538       $unwind$Java_NotifyFramePopStressTest_suspend 0000000180004538     libNotifyFramePopStressTest.obj
 0002:00001538       $unwind$__raise_securityfailure 0000000180004538     MSVCRT:gs_report.obj
 0002:00001538       $unwind$_Init_thread_footer 0000000180004538     MSVCRT:thread_safe_statics.obj
 0002:00001538       $unwind$_Init_thread_header 0000000180004538     MSVCRT:thread_safe_statics.obj
 0002:00001538       $unwind$_Init_thread_wait  0000000180004538     MSVCRT:thread_safe_statics.obj
 0002:00001538       $unwind$__scrt_initialize_crt 0000000180004538     MSVCRT:utility.obj
 0002:00001538       $unwind$__scrt_initialize_onexit_tables 0000000180004538     MSVCRT:utility.obj
 0002:00001538       $unwind$__scrt_release_startup_lock 0000000180004538     MSVCRT:utility.obj
 0002:00001538       $unwind$__scrt_uninitialize_crt 0000000180004538     MSVCRT:utility.obj
 0002:00001538       $unwind$_onexit            0000000180004538     MSVCRT:utility.obj
 0002:00001540       $unwind$?print_stack_trace@@YAXPEAU_jvmtiEnv@@PEAUJNIEnv_@@PEAV_jobject@@@Z 0000000180004540     libNotifyFramePopStressTest.obj
 0002:00001560       $unwind$Agent_Initialize   0000000180004560     libNotifyFramePopStressTest.obj
 0002:00001560       $unwind$__scrt_initialize_default_local_stdio_options 0000000180004560     MSVCRT:default_local_stdio_options.obj
 0002:00001560       $unwind$?dllmain_crt_dispatch@@YAHQEAUHINSTANCE__@@KQEAX@Z 0000000180004560     MSVCRT:dll_dllmain.obj
 0002:00001560       $unwind$DllMain            0000000180004560     MSVCRT:dll_dllmain_stub.obj
 0002:00001560       $unwind$__GSHandlerCheck   0000000180004560     MSVCRT:gshandler.obj
 0002:00001560       $unwind$?__scrt_uninitialize_thread_safe_statics@@YAXXZ 0000000180004560     MSVCRT:thread_safe_statics.obj
 0002:00001560       $unwind$_Init_thread_notify 0000000180004560     MSVCRT:thread_safe_statics.obj
 0002:00001560       $unwind$__scrt_acquire_startup_lock 0000000180004560     MSVCRT:utility.obj
 0002:00001560       $unwind$__scrt_dllmain_after_initialize_c 0000000180004560     MSVCRT:utility.obj
 0002:00001560       $unwind$__scrt_dllmain_before_initialize_c 0000000180004560     MSVCRT:utility.obj
 0002:00001560       $unwind$__scrt_dllmain_crt_thread_attach 0000000180004560     MSVCRT:utility.obj
 0002:00001560       $unwind$__scrt_dllmain_crt_thread_detach 0000000180004560     MSVCRT:utility.obj
 0002:00001560       $unwind$__scrt_dllmain_uninitialize_c 0000000180004560     MSVCRT:utility.obj
 0002:00001560       $unwind$__scrt_dllmain_uninitialize_critical 0000000180004560     MSVCRT:utility.obj
 0002:00001560       $unwind$atexit             0000000180004560     MSVCRT:utility.obj
 0002:00001568       $unwind$FramePop           0000000180004568     libNotifyFramePopStressTest.obj
 0002:00001578       $unwind$Java_NotifyFramePopStressTest_notifyFramePop 0000000180004578     libNotifyFramePopStressTest.obj
 0002:0000158c       $unwind$_RTC_Initialize    000000018000458c     MSVCRT:initsect.obj
 0002:0000158c       $unwind$_RTC_Terminate     000000018000458c     MSVCRT:initsect.obj
 0002:0000158c       $unwind$?__scrt_initialize_thread_safe_statics@@YAHXZ 000000018000458c     MSVCRT:thread_safe_statics.obj
 0002:00001598       $unwind$__GSHandlerCheckCommon 0000000180004598     MSVCRT:gshandler.obj
 0002:000015a0       $xdatasym                  00000001800045a0     MSVCRT:amdsecgs.obj
 0002:000015a4       $unwind$?dllmain_crt_process_attach@@YAHQEAUHINSTANCE__@@QEAX@Z 00000001800045a4     MSVCRT:dll_dllmain.obj
 0002:000015e0       $unwind$?fin$0@?0??dllmain_crt_process_attach@@YAHQEAUHINSTANCE__@@QEAX@Z@4HA 00000001800045e0     MSVCRT:dll_dllmain.obj
 0002:000015e0       $unwind$?fin$0@?0??dllmain_crt_process_detach@@YAH_N@Z@4HA 00000001800045e0     MSVCRT:dll_dllmain.obj
 0002:000015e0       $unwind$?fin$1@?0??dllmain_crt_process_detach@@YAH_N@Z@4HA 00000001800045e0     MSVCRT:dll_dllmain.obj
 0002:000015e8       $unwind$?dllmain_crt_process_detach@@YAH_N@Z 00000001800045e8     MSVCRT:dll_dllmain.obj
 0002:0000163c       $unwind$?dllmain_dispatch@@YAHQEAUHINSTANCE__@@KQEAX@Z 000000018000463c     MSVCRT:dll_dllmain.obj
 0002:00001664       $unwind$?filt$0@?0??dllmain_dispatch@@YAHQEAUHINSTANCE__@@KQEAX@Z@4HA 0000000180004664     MSVCRT:dll_dllmain.obj
 0002:0000166c       $unwind$_DllMainCRTStartup 000000018000466c     MSVCRT:dll_dllmain.obj
 0002:0000167c       $unwind$__scrt_is_nonwritable_in_current_image 000000018000467c     MSVCRT:utility.obj
 0002:0000169c       $unwind$__scrt_is_nonwritable_in_current_image$filt$0 000000018000469c     MSVCRT:utility.obj
 0002:000016a4       $unwind$__scrt_dllmain_exception_filter 00000001800046a4     MSVCRT:utility.obj
 0002:000016b8       $unwind$__scrt_fastfail    00000001800046b8     MSVCRT:utility_desktop.obj
 0002:000016c8       $unwind$__report_gsfailure 00000001800046c8     MSVCRT:gs_report.obj
 0002:000016d0       $unwind$capture_previous_context 00000001800046d0     MSVCRT:gs_report.obj
 0002:000016dc       $unwind$__security_init_cookie 00000001800046dc     MSVCRT:gs_support.obj
 0002:000016e8       $unwind$__isa_available_init 00000001800046e8     MSVCRT:cpu_disp.obj
 0002:000016f8       $xdatasym                  00000001800046f8     MSVCRT:guard_dispatch.obj
 0002:00001700       $xdatasym                  0000000180004700     MSVCRT:guard_xfg_dispatch.obj
 0002:00001710       .edata                     0000000180004710     NotifyFramePopStressTest.exp
 0002:00001738       rgpv                       0000000180004738     NotifyFramePopStressTest.exp
 0002:00001760       rgszName                   0000000180004760     NotifyFramePopStressTest.exp
 0002:00001788       rgwOrd                     0000000180004788     NotifyFramePopStressTest.exp
 0002:0000179c       szName                     000000018000479c     NotifyFramePopStressTest.exp
 0002:000017b9       $N00001                    00000001800047b9     NotifyFramePopStressTest.exp
 0002:000017c8       $N00002                    00000001800047c8     NotifyFramePopStressTest.exp
 0002:000017d5       $N00003                    00000001800047d5     NotifyFramePopStressTest.exp
 0002:000017e0       $N00004                    00000001800047e0     NotifyFramePopStressTest.exp
 0002:00001818       $N00005                    0000000180004818     NotifyFramePopStressTest.exp
 0002:0000183d       $N00006                    000000018000483d     NotifyFramePopStressTest.exp
 0002:00001867       $N00007                    0000000180004867     NotifyFramePopStressTest.exp
 0002:00001894       $N00008                    0000000180004894     NotifyFramePopStressTest.exp
 0002:000018b9       $N00009                    00000001800048b9     NotifyFramePopStressTest.exp
 0002:000018f3       $N00010                    00000001800048f3     NotifyFramePopStressTest.exp
 0002:00001d84       .idata$6                   0000000180004d84     kernel32:KERNEL32.dll
 0002:00001dd4       .idata$6                   0000000180004dd4     vcruntime:VCRUNTIME140.dll
 0002:00001f12       .idata$6                   0000000180004f12     ucrt:api-ms-win-crt-stdio-l1-1-0.dll
 0002:00001f32       .idata$6                   0000000180004f32     ucrt:api-ms-win-crt-string-l1-1-0.dll
 0002:00001f54       .idata$6                   0000000180004f54     ucrt:api-ms-win-crt-runtime-l1-1-0.dll
 0003:00000000       ?UNNAMED_STR@?1??get_thread_name@@YAPEADPEAU_jvmtiEnv@@PEAUJNIEnv_@@PEAV_jobject@@@Z@4PEBDEB 0000000180005000     libNotifyFramePopStressTest.obj
 0003:00000058       ?UNNAMED_LEN@?1??get_thread_name@@YAPEADPEAU_jvmtiEnv@@PEAUJNIEnv_@@PEAV_jobject@@@Z@4_KA 0000000180005058     libNotifyFramePopStressTest.obj
 0003:00000060       ?$TSS0@?1??get_thread_name@@YAPEADPEAU_jvmtiEnv@@PEAUJNIEnv_@@PEAV_jobject@@@Z@4HA 0000000180005060     libNotifyFramePopStressTest.obj
 0003:00000070       jvmti                      0000000180005070     libNotifyFramePopStressTest.obj
 0003:00000078       caps                       0000000180005078     libNotifyFramePopStressTest.obj
 0003:00000088       pop_count                  0000000180005088     libNotifyFramePopStressTest.obj
 0003:0000008c       failed                     000000018000508c     libNotifyFramePopStressTest.obj
 0003:0000008d       seenMain                   000000018000508d     libNotifyFramePopStressTest.obj
 0003:00000090       callbacks                  0000000180005090     libNotifyFramePopStressTest.obj
 0003:000001c8       last_notify_method         00000001800051c8     libNotifyFramePopStressTest.obj
 0003:000001d0       ?g_tss_cv@@3U_RTL_CONDITION_VARIABLE@@A 00000001800051d0     MSVCRT:thread_safe_statics.obj
 0003:000001d8       ?g_tss_event@@3PEAXEA      00000001800051d8     MSVCRT:thread_safe_statics.obj
 0003:000001e0       ?g_tss_mutex@@3U_RTL_CRITICAL_SECTION@@A 00000001800051e0     MSVCRT:thread_safe_statics.obj
 0003:00000208       ?g_sleep_condition_variable_cs@@3P6AHPEAU_RTL_CONDITION_VARIABLE@@PEAU_RTL_CRITICAL_SECTION@@K@ZEA 0000000180005208     MSVCRT:thread_safe_statics.obj
 0003:00000210       ?g_wake_all_condition_variable@@3P6AXPEAU_RTL_CONDITION_VARIABLE@@@ZEA 0000000180005210     MSVCRT:thread_safe_statics.obj
 0003:0000021c       ?__proc_attached@@3HA      000000018000521c     MSVCRT:dll_dllmain.obj
 0003:00000230       ?is_initialized_as_dll@@3_NA 0000000180005230     MSVCRT:utility.obj
 0003:00000231       ?module_local_atexit_table_initialized@@3_NA 0000000180005231     MSVCRT:utility.obj
 0003:00000238       ?module_local_atexit_table@@3U_onexit_table_t@@A 0000000180005238     MSVCRT:utility.obj
 0003:00000250       ?module_local_at_quick_exit_table@@3U_onexit_table_t@@A 0000000180005250     MSVCRT:utility.obj
 0003:00000270       GS_ExceptionRecord         0000000180005270     MSVCRT:gs_report.obj
 0003:00000310       GS_ContextRecord           0000000180005310     MSVCRT:gs_report.obj
